:100000002030840025300C208316FF2390008301CC
:10001000B02B04068001840A0406031D092864002D
:020020000034AA
:100760008312FF2383169000831285013B3083168A
:100770008500073083129900133083169F000130E3
:1007800083129F00051AC22B1F150730A400A40B6B
:10079000C72B9F149F18CA2B1E08A2001F110730D9
:1007A000A400A40BD12B9F149F18D42B1E08A000CB
:1007B000051A851EDD2B0310A20C051E851EE12BDC
:1007C000A201051AE52B851EED2B22082302031C2E
:1007D000A30A23082202031CA303A0080319C42BA5
:1007E000A003FF30A100A1080319ED2BA1032308EA
:0E07F00021020318FD2B0515F32B0511F32B29
:02400E00E43F8D
:00000001FF
